:1000000012C0189518951895189518951895189563
:1000100077C0E2C0189518951895189518951895F9
:100020001895189518958FE58DBFC0EEE8E64E2E11
:1000300084E08EBFD3E0F3E05F2EEEEFF3E0A0E6C6
:10004000B0E084B7082E877F84BF8FE181BD80E058
:1000500081BD88278D933197E9F7EDD0662483E23F
:100060008093620080E08FBD84E08EBDE4D084E6A2
:1000700090E061D18CE033D1CAD0B89A89B784605E
:1000800089BF78947ED08FE711E0D0D0EEE1F5E023
:10009000B8D08FEB11E0CAD0E0E3F5E0B2D05AD18E
:1000A000A0E6B0E02C93A1E6B0E01C9300916000C4
:1000B0000F3F09F424C0A1E6B0E08C918F778C93B8
:1000C000A6D08FE711E0B2D0E2E4F5E09AD08FE756
:1000D0001AE0ACD0E8E4F5E094D08FEB11E0A6D0C4
:1000E000A0E5B3E0E0E6F0E0D0D183D08FEB1AE0FA
:1000F0009DD0A0E5B3E0E1E6F0E0C7D17AD0CFCF64
:100100000F921F922F923F924F925F927F92AF92E7
:10011000BF920F931F932F933F934F935F936F93D0
:100120007F938F939F93AF93BF93CF93DF93EF937F
:10013000FF938FB78F938EEE95E890934D00809349
:100140004C0088B391E0892788BB8F918FBFFF91C6
:10015000EF91DF91CF91BF91AF919F918F917F915F
:100160006F915F914F913F912F911F910F91BF9090
:10017000AF907F905F904F903F902F901F900F9087
:100180001895009162004FE00423A3E6B0E00C93C1
:10019000A3E6B0E08C9180598C93809162008093AB
:1001A000640094E0A4E6B0E047D1A4E6B0E08C910E
:1001B00083708C93A4E6B0E08C918C5A8C9389E286
:1001C0008ED0809163008BD08091640088D088E2CB
:1001D00086D00895F894FFCF8F939F938FB7339570
:1001E000539509F4439591EC92BF9F918FBF8F91E6
:1001F0001895A0E5B3E08D91882311F06AD0FBCF6C
:10020000089522D1802D11F064D0FBCF089581E0B4
:1002100066D00ED080E863C08FE7213039F08FEBD5
:10022000223021F08FE8233009F08FEC810F57C086
:1002300083E0992780C08AEF90E07DD0A39AA29AAC
:10024000A19AA09AA49AA59AAD9885E090E073D05F
:10025000AC98AB98AA98A99AA89AAC9AEF93FF93F6
:10026000E4ECF0E05CD0FF91EF91AC9861D0AC9AF7
:10027000EF93FF93E4ECF0E052D0FF91EF91AC9854
:1002800057D0AC9AEF93FF93E4ECF0E048D0FF91A5
:10029000EF91AC984DD0A898AC9AEF93FF93E4EC13
:1002A000F0E03DD0FF91EF91AC9842D089E217D0B9
:1002B0008CE115D082E513D089E611D084E70FD008
:1002C00088E20DD088E20BD08EE009D086E007D01E
:1002D0000895AD9A829505D004D02AD00895AD989E
:1002E000F9CF859510F4A89A01C0A898859510F4C7
:1002F000A99A01C0A998859510F4AA9A01C0AA9854
:10030000859510F4AB9A01C0AB98AC9AEF93FF932C
:10031000E4ECF0E004D0FF91EF91AC9808953197B0
:10032000F1F70895689462F80895E89462F80895E2
:1003300081E090E000C0EF93FF93EE27E82BE92BDC
:1003400031F0E0EDF7E03197F1F70197D1F7FF9148
:10035000EF9108950F933F934F935F932F923F92A6
:100360008F939F938FB78F9383B78F93826083BF51
:1003700089B78F93816089BF81EC82BF552744275D
:100380003327483008F047C0373324F4879BF8CF31
:10039000F8CF41C04830ECF78799FCCF3327323291
:1003A000D4F5879BFCCF932F332711272227913138
:1003B00010F0969511E0292E2694322C290E990FD3
:1003C000390E113021F0321534F58799FCCF3327DF
:1003D0000CE03215F0F3879909C08894111F221F91
:1003E0003315CCF4879BFCCF332708C00894111F2A
:1003F000221F331584F48799FCCF33270A9549F7D8
:10040000912F991F221F991F221F25FB17F926FBE9
:1004100016F92F7102C01FEF2FEF8F9189BF8F91B7
:1004200083BF8F918FBF9F918F913F902F905F914E
:100430004F913F910F910895903029F08C918695BE
:100440009A95E9F78C930895C89531960020089500
:10045000000F111F221F331F08950095109520953E
:1004600030950F5F1F4F2F4F3F4F0895019110811F
:100470000EC001911191219130810BC00191108129
:1004800017FF05C03FEF2FEF04C00081112722277F
:10049000332737FF03C0E1DF8DE28D93CF93DF93E6
:1004A000CF92DF92EF92AA24BB24CC24DD24EE2449
:1004B00040E2CAE0DD2755E093E38881890F87FD9C
:1004C0009F7083FD907F891B89935A95A9F7C0DFA0
:1004D000AA1CBB1CCC1CDD1CEE1C4A9551F7E894F1
:1004E000EFE0FF2782910ED0EB30E0F71EF068942A
:1004F0008A2D0CD088278D93EF90DF90CF90DF91DD
:10050000CF910895982F829501D0892F8F70805DAB
:1005100026F0803309F4089568948D9308952A5243
:1005200043352D456D706661656E6765722A000002
:1005300057616974696E6720666F72205243352176
:0E05400000004144523A0000434F4D3A000083
:00000001FF
